:020000040000FA
:0400000069303A2801
:08000800A000030EA100831209
:1000100005191028831601178312B23081002B288E
:1000200083160113831203140B190310A80DA90DD5
:10003000AA0DAB0DAC0DAC16FF302C02031D2B2806
:10004000FA302B02031D2B2831152A08AF0029088E
:10005000AE002808AD008B100B11210E8300A00EFE
:04006000200E090065
:0C007400203084008001840A80300402E7
:10008000031C3C281230B000342283160C30850546
:1000900087018312850187010730990000309A009B
:1000A000103083168E008312603083168F00831207
:1000B0000030831691009F008312C83083168100A0
:1000C000831231309000003083168C008312103080
:1000D0008B00BC1B7128851971286400851D6D2853
:1000E000D0233C1C7428312381018E018F010B1118
:1000F0008B100B108C018B178C2031198F2016223E
:10010000B30B8A28031085190314B90DF030390296
:100110000319972142237C28640032100800311112
:100120000130B70085144008013ECE000F08CF0013
:100130008B132030370783169B001C141A08831278
:10014000A4001030370783169B001C141A08831272
:10015000A300A6000230A6060030370783169B00D6
:100160001C141A088312A200A7000130A7068B17DF
:10017000321CC02822090339A200A309A409A50939
:1001800024082F02031D912923082E02031D2A296A
:1001900022082D02031D912901303702031DD728A3
:1001A0003C19D6283D18D7283D143E145122023060
:1001B0003702031DE2283C19E128BD18E228BD14CE
:1001C0003E145E2203303702031DED283C19EC2853
:1001D0003D19ED283D153E146B2204303702031DF6
:1001E000F8283C19F728BD19F828BD153E147822C7
:1001F00005303702031D03293C1902293D1A032942
:100200003D163E14852206303702031D0E293C1987
:100210000D29BD1A0E29BD163E1492220730370251
:10022000031D19293C1918293D1B19293D173E1496
:100230009F2208303702031D24293C192329BD1BA6
:100240002429BD173E14AC2209303702031D2A2988
:100250003E14B92226082E02031D912927082D02DB
:10026000031D912901303702031D3D293C193C290A
:100270003D1C3D293D103E14E02202303702031D93
:1002800048293C194729BD1C4829BD103E14E422C9
:1002900003303702031D53293C1952293D1D5329B0
:1002A0003D113E14E82204303702031D5E293C193B
:1002B0005D29BD1D5E29BD113E14EC2205303702BB
:1002C000031D69293C1968293D1E69293D123E1408
:1002D000F02206303702031D74293C197329BD1E14
:1002E0007429BD123E14F42207303702031D7F2902
:1002F0003C197E293D1F7F293D133E14F82208300A
:100300003702031D8A293C198929BD1F8A29BD137B
:100310003E14FC2209303702031D90293E140023AD
:100320009129B70A0A3037020318080098280130CB
:10033000B600B300B400B500B70085018701B11362
:100340008C20B30BDD29031085190314B90DF0308F
:1003500039020319042AB41F8510B40BDD290130BA
:10036000370203190423023037020319082303302C
:10037000370203190C230430370203191023053008
:1003800037020319142306303702031918230730E4
:10039000370203191C2308303702031920230930C0
:1003A0003702031924233708B6080319B6000319C6
:1003B000DB298514B6039630B400311DA029311114
:1003C000321CE7292D090339AD00AE09AF092F1CF6
:1003D000A0298E018F010C1CA0290C102E1EA02913
:1003E0008B1320303707BB002F08BA001F221030B4
:1003F0003707BB002E08BA001F2200303707BB00AA
:100400002D08BA001F228B1785018701083037029B
:100410002030031985002A3003198700B70AB60176
:100420000A303702031CA029312308003E1C0800B3
:100430003E101030BB003D08BA001F2208008B138D
:100440003A0883161C159A0083123B0883169B00FA
:1004500055309D00AA309D009C1464009C182D2AE4
:100460001C1183128B170800831600309B001C148C
:100470001A088312BC00831610309B001C141A0843
:1004800083123C18BD00831620309B001C141A08F0
:100490008312C1000130C11BC100C1080319C10092
:1004A00008003C19871640083C1D40034107D00056
:1004B0000F08D100BC192B233D1408003C19071666
:1004C00040083C1D40034107D2000F08D300BC196F
:1004D0002B23BD1408003C19871540083C1D400320
:1004E0004107D4000F08D500BC192B233D15080087
:1004F0003C19051640083C1D40034107D6000F0873
:10050000D700BC192B23BD1508003C1985164008DF
:100510003C1D40034107D8000F08D900BC192B230C
:100520003D1608003C19071540083C1D40034107D3
:10053000DA000F08DB00BC192B23BD1608003C199C
:10054000871440083C1D40034107DC000F08DD0014
:10055000BC192B233D1708003C19071440083C1D0B
:1005600040034107DE000F08DF00BC192B23BD1735
:100570000800BC1908003C1DC12A303085043F30FA
:1005800087048E018F01C001D001D201D401D601B0
:100590000130D800DA00DC00DE004030D1008030CD
:1005A000D300C030D500FF30D7004030D9008030B4
:1005B000DB00C030DD00FF30DF00FF30BD00080091
:1005C00087128E018F01080007128E018F0108002B
:1005D00087118E018F01080005128E018F0108001E
:1005E00085128E018F01080007118E018F0108000E
:1005F00087108E018F01080007108E018F010800FF
:100600002B238E018F0108000708203A870008007D
:100610000708103A870008000708083A8700080012
:100620000508103A850008000508203A85000800F2
:100630000708043A870008000708023A8700080004
:100640000708013A870008000508303A85000708C6
:100650003F3A87000800CF308505C0308705BD01CF
:1006600008003D188716BD1807163D198715BD19D6
:1006700005163D1A8516BD1A07153D1B8714BD1BAF
:10068000071408003C19462B3D1C522B5008400211
:10069000031D522B51080F02031C522B3C198712C9
:1006A0003C1D87163C19562BBD1C622B520840027C
:1006B000031D622B53080F02031C622B3C19071207
:1006C0003C1D07163C19662B3D1D722B5408400239
:1006D000031D722B55080F02031C722B3C19871146
:1006E0003C1D87153C19762BBD1D822B56084002F8
:1006F000031D822B57080F02031C822B3C19051285
:100700003C1D05163C19862B3D1E922B58084002B5
:10071000031D922B59080F02031C922B3C198512C2
:100720003C1D85163C19962BBD1EA22B5A08400273
:10073000031DA22B5B080F02031CA22B3C190711FF
:100740003C1D07153C19A62B3D1FB22B5C0840022F
:10075000031DB22B5D080F02031CB22B3C1987103E
:100760003C1D87143C19B62BBD1FC22B5E084002EE
:10077000031DC22B5F080F02031CC22B3C1907107C
:100780003C1D07144E084002031DCB2B4F080F02DF
:10079000031CCB2B85100C1C08000C10C00A080091
:1007A000B601B301B4013C1CD82BBC01BC14E42B32
:1007B000BC1CDD2BBC013C15E42B3C1DE22BBC0119
:1007C000BC15E42BBC013C143C08B6006400E82BCB
:1007D000E92BEA2BEB2BEC2BB41B8716B41F8712EB
:1007E000B30BE62BB40BE62B0310B60CB608031DB7
:0E07F000E62B0030BB003C08BA001F220800B8
:084000000800030006000500A2
:02400E00CC33B1
:10420000010078007A007C007E007B0079007F004E
:104210007D007A0078007E007C00FF00FF00FF0038
:104220000000F200F600FA00FE00F200F600FA00CC
:10423000FE00F200F600FA00FE00FF00FF00FF00A3
:10424000010005000500050005000900090009003E
:1042500009000D000D000D000D00FF00FF00FF0024
:10426000FF00FF00FF00FF00FF00FF00FF00FF0056
:10427000FF00FF00FF00FF00FF00FF00FF00FF0046
:10428000FF00FF00FF00FF00FF00FF00FF00FF0036
:10429000FF00FF00FF00FF00FF00FF00FF00FF0026
:1042A000FF00FF00FF00FF00FF00FF00FF00FF0016
:1042B000FF00FF00FF00FF00FF00FF00FF00FF0006
:1042C000FF00FF00FF00FF00FF00FF00FF00FF00F6
:1042D000FF00FF00FF00FF00FF00FF00FF00FF00E6
:1042E000FF00FF00FF00FF00FF00FF00FF00FF00D6
:1042F000FF00FF00FF00FF00FF00FF00FF00DD00E8
:00000001FF
